:020000040000FA
:1000000007309F008501860183168111F03085003D
:1000100086019B011C141A088312850083169B0A13
:100020001C14831286008E11F030640085050319BC
:1000300015288E15051A3128851A4928051B6128AF
:1000400079281930A1008430A000A00B2528A10B2D
:1000500023280800640021200508F039031908004E
:100060002A2885150518362805147B2806183A28ED
:1000700006147B2886183F28861406107B28051056
:100080000610861085187B2805197B288511861394
:100090009428851585184E2885147B280619522822
:1000A00006157B2886195728861506117B2885108A
:1000B0000611861105187B2805197B2885118613E2
:1000C000942885150519662805157B28061A6A28BF
:1000D00006167B28861A6F28861606127B280511BD
:1000E0000612861205187B2885187B288511861331
:1000F0009428803086068618832886198328861AD5
:10010000832886179428861C8B28861D8E28861E99
:1001100091288613942805189428852885189428F2
:10012000872805199428892805088C1383169B01B4
:100130009A001C1555309D00AA309D009C141C117E
:10014000831206088C1BA6286400A2288C13831631
:100150009B0A9A001C1555309D00AA309D009C14E6
:100160001C1183128C1BB6286400B2282A20132885
:02400E0014029A
:00000001FF
